:0600000000008A01002946
:08000800F000030EF1000B1DD6
:1000100033280B11F20A7208083C031D2E28F20146
:100020008B1000000000000000000B16F30A73089C
:100030000A3C031D2C28F70AF301F60AF40A740897
:10004000063C031D2C28F401F50A7508033C031D2A
:100050002C28F501F601F60AFA0A41287208043C38
:100060000319F90A41288B1C00298B100B128101FE
:1000700000000B11F201F301F401F501F601F60A9B
:0C008000F70A710E8300F00E700E0900EC
:1001000082070134413400340034013400340034B7
:1001100000340134813410340034013400340034AC
:1001200000340234113450340034013400340034CB
:1001300000340234493430340034013400340034A3
:10014000003402348234003400340134003400348A
:02015000003479
:02016E00820706
:0C0170000034203408340434023401341C
:02017E008207F6
:1001800000340034003400340134003400340234CC
:1001900000340034043400340034083400340034B3
:1001A00000340134003400340234003400340434A8
:1001B0000034003408340034103400340034203467
:1001C000003400340034103400340034203400345F
:1001D00000344034003400348034023400340034BD
:1001E000043400340034103400340034203400343B
:0201F0000034D9
:100200008B0183130313831264008316BF308100B4
:1002100006309F00FF308500860087008800890136
:100220008C018D0103178C0183128C018E018D01CD
:100230008F0103139701900192018C018D019F01A1
:100240008901F201F301F401F501F601F60AF70163
:10025000F801F901FA01A501A601F801A301A10124
:10026000A20183160C309900203098008312803050
:100270009800861F362A061F9A2985018601870164
:10028000880186194929363086003F308700FF30C3
:1002900088008316C9308600C0308700003088008F
:1002A00083120B168B168B17F70A2124F808031DEF
:1002B0006329F708031D7D29F908031D9629FA080B
:1002C000031D98295529F8012408A600031D6D294E
:1002D000A20157240301142455297603AC002603F8
:1002E0002C02031C123E013EA2005724A40E240D32
:1002F000A40EE039220714245529F701A608031D8E
:100300008629A20157240301142455297603AC0041
:1003100026032C02031C123E013EA2005724A40E09
:10032000240DA40EE039220714245529F90155297A
:10033000FA01552985018601870188018316C93094
:100340008600C03087000030880083120B168B16A1
:100350008B17F70ABF243124A408031DB62987127E
:100360000712880186010301861D14242124F80840
:10037000031DDD29F708031DFF29F908031D192AAC
:10038000FA08031D222A260823020319B629260883
:10039000A3000319B629861DB6292603A900A90DB5
:1003A000A90D290DF839A9000530AA0029088020D7
:1003B0001424A90AAA0BD629B629F801A6080319FC
:1003C000BF242408A600031DEE29A20187120712EC
:1003D000880186010301861D1424B6297603AC002A
:1003E00026032C02031C123E013EA200A40E240D83
:1003F000A40EE0392207861D14248124222AF70145
:10040000A608031D082AA2010301861D1424B6298B
:100410007603AC0026032C02031C123E013EA20010
:10042000A40E240DA40EE0392207861D1424812475
:10043000222AF901A6080319B629CD30E724203075
:10044000F224B629FA01A6080319B629CC30E7240C
:100450008B137508303EF2243A30F2247408303E93
:10046000F2247308303EF2248B17B62985018601E9
:10047000870188018619442A2F308500363086008E
:100480003F308700FF3088008316D0308500C930A8
:100490008600C030870000308800831218168C1A3E
:1004A0005C2A0000000000000000000000000000C6
:1004B0000000000000004F2A1808AB001A08A00036
:1004C000AB1C652A1812000018162B194F2A200899
:1004D0001F39A200A00E200CA00E0739A100432452
:1004E00057242108230203194F2A2108A3000319C6
:1004F0004F2A2103A900A90DA90D290DF839A9003A
:100500000530AA00290880201424A90AAA0B822AEF
:020510004F2A70
:10080000A701A801A80B022CA70B022C0800193085
:10081000A700A80100000000000000000000A80BD5
:100820000A2CA70B0A2C0800AD010C1A1F2C000083
:100830000000000000000000AD0B152CFF349900F3
:1008400000343124240826020319302C2408250200
:1008500003192F2C2408A50007243124262CF80A7C
:1008600008000530A400051C0800A403851C08002E
:10087000A403051D0800A403851D0800A403851E0C
:100880000800A40308002108073A0319522C063077
:1008900021020319080021088A01B720861D2F3A7A
:1008A000850008002F30861D2F3A85000800220899
:1008B0001F3A0319742C2208123C031C080022085A
:1008C00022072207AC008A01BF20861D363A860027
:1008D0002C0ABF20861D3F3A8700AC0A2C0ABF2095
:1008E000861DFF3A880008003630861D363A86009D
:1008F0003F30861D3F3A8700FF30861DFF3A880053
:1009000008002203A900A90DA90D290DF839A90095
:100910000830AA008030E72406308A0029080F2614
:10092000F224A90AAA0B8E2C2030F2242030F224C3
:100930002603A900A90DA90D290DF839A900063033
:10094000AA0006308A002908BF26F224A90AAA0BA9
:10095000A32C2203A900A907A907A9072908290789
:10096000A9070C30AA00C030E72407308A00290804
:100970000F27F224A90AAA0BB72C8A010800061235
:1009800086140724061500243830E724072438305D
:10099000E724A80100000000000000000000A80BF0
:1009A000CA2C3830E724A801000000000000000035
:1009B0000000A80BD42C3830E7240830E7240025A9
:1009C0000630E7240C30E72410258616080088003E
:1009D00000000716000007121430AE008801AE0BAD
:1009E000EF2C080088008716000007160000071289
:1009F000000087121430AE008801AE0BFD2C0800F9
:100A0000013088000000071600000712A8018801C5
:100A100000000000000000000000A80B082D0800E6
:100A2000023088000000071600000712A8018801A4
:100A300000000000000000000000A80B182D0800B6
:020C1E0082074B
:100C200034345534313455344E3420342034203467
:100C3000563445343834413454342034203420344C
:100C40005734363457345834203420342034203448
:100C50004B344834363457344F3420342034203425
:100C60005A344C3436344234203420342034203446
:100C700056344B34363452344234503420342034D9
:100C80004A344134323449344734593420342034DE
:100C90005234523439344F34203420342034203408
:100CA0005634523432344234203420342034203408
:100CB0003434533437344234203420342034203414
:100CC0005A345334363444344E34203420342034AF
:100CD00035345A34343442342034203420342034EF
:100CE0003434583436345434553420342034203499
:100CF0004F344834323442342034203420342034C9
:100D000043345334333442342034203420342034B8
:100D10004C3455343434413441342034203420347C
:100D20004F3441343434423420342034203420349D
:100D3000593456343534423420342034203420346D
:020D7E008207EA
:100D8000313434342E34313430343034203420345F
:100D9000313438342E34313431343034203420344A
:100DA000323431342E34313435343034203420343C
:100DB000323434342E343934333430342034203423
:100DC000323438342E343234303430342034203419
:020E1E00820749
:100E20004E3465347734203459346F3472346B3433
:100E30002034203420342034433461346E3461341F
:100E4000643461342034203420342034203420347D
:100E5000433461346C34693466346F3472346E34C4
:100E60006934613420342034483461347734613457
:100E70006934693420342034203420342034203440
:100E80004E346534773420345A34653461346C34EC
:100E900061346E34643420344134753473347434C2
:100EA000723461346C346934613420342034203439
:100EB0004A346134703461346E3420342034203448
:100EC0002034203420342034523475347334733455
:100ED00069346134203420342034203420342034E8
:100EE00048346F346E34673420344B346F346E348E
:100EF000673420342034203453347234693420343D
:100F00004C3461346E346B346134203420342034FA
:100F100053342E34203441346634723469346334AB
:100F200061342034203420344B3465346E347934C9
:100F300061342034203420342034203420342034D0
:100F4000493473347234613465346C342034203461
:100F50002034203420342034463469346E346C34E8
:100F600061346E346434203420342034203420340E
:100F70004D346134643465346934723461342034FE
:100F800020342034203420344134723467346534C2
:100F90006E34743469346E34613420342034203437
:100FA0005034653472347534203420342034203485
:100FB0002034203420342034563465346E34653483
:100FC0007A34753465346C34613420342034203400
:02400E00313D42
:00000001FF
